:1000000012C029C040C027C026C025C025C023C0BB
:1000100022C021C020C01FC01EC01DC01CC01BC0EC
:100020001AC019C018C011241FBECFEDCDBF10E0FB
:10003000A0E6B0E0E8EEF2E002C005900D92A03636
:10004000B107D9F710E0A0E6B0E001C01D92AC36D0
:10005000B107E1F778C0D4CF1F920F920FB60F927D
:1000600011248F939F938091640090916500019675
:1000700090936500809364009F918F910F900FBEC5
:100080000F901F9018951F920F920FB60F92112488
:100090002F933F934F935F938F939F93AF93BF9310
:1000A00022B78091640090916500982F8827820F75
:1000B000911DAA27BB278093600090936100A093B5
:1000C0006200B09363002091600030916100409124
:1000D0006200509163008091660090916700A0914A
:1000E0006800B0916900281739074A075B0780F458
:1000F0008091600090916100A0916200B0916300D6
:100100008093660090936700A0936800B0936900A5
:1001100012BE109265001092640080916A00909166
:100120006B00019690936B0080936A00BF91AF9132
:100130009F918F915F914F913F912F910F900FBEA3
:100140000F901F901895CFEDD0E0DEBFCDBFBB9ACA
:1001500089B7826089BF85B7846085BF8BB78068A7
:100160008BBF83B7816083BF7894839991C0C39A12
:1001700012BE109265001092640010926B001092F3
:100180006A008FEF9FEFA0E0B0E08093660090934D
:100190006700A0936800B093690080916A00909115
:1001A0006B00099708F050C082B72091640030912D
:1001B0006500A0906600B0906700C0906800D09085
:1001C0006900D694C794B794A794D694C794B7946B
:1001D000A794E0906600F09067000091680010918D
:1001E0006900322F2227280F311D44275527C501CA
:1001F000AA2797FDA095BA2F8E0D9F1DA01FB11F96
:10020000281739074A075B0740F280916A009091EE
:100210006B00019690936B0080936A00C50160E0CB
:1002200071E03BD082BFC501B7FC34C0892F990F64
:10023000990B909365008093640080916A0090917F
:100240006B00099708F4B0CF839BFECF62E070E0AB
:1002500082B72091640030916500E0906600F090D4
:1002600067000091680010916900322F2227280F43
:10027000311D44275527E216F3060407150710F031
:100280008399E6CF6150704077FFE2CF839B6FCFB9
:10029000C3986BCF81509F4FC9CF97FB092E07267C
:1002A0000AD077FD04D00CD006D000201AF4709547
:1002B00061957F4F0895F6F7909581959F4F08952A
:1002C000AA1BBB1B51E107C0AA1FBB1FA617B7077C
:1002D00010F0A61BB70B881F991F5A95A9F7809598
:0802E0009095BC01CD010895C9
:00000001FF
